:100000000C942A000C9445000C9445000C94450077
:100010000C9445000C9445000C9445000C9445004C
:100020000C9445000C9445000C9445000C9445003C
:100030000C9445000C9445000C9445000C9445002C
:100040000C9445000C9445000C9445000C9445001C
:100050000C94450011241FBECFE5D4E0DEBFCDBF18
:1000600010E0A0E6B0E0E6ECF0E002C005900D92F2
:10007000A036B107D9F710E0A0E6B0E001C01D92AC
:10008000A036B107E1F70C9447000C940000CFE5CF
:10009000D4E0DEBFCDBF1BB888E18AB984E880BD5B
:1000A00010BC87E189B95F9BFECF8BB199278C711A
:1000B0009070892B19F08CB18FE301C08CB15D9BDE
:0600C000FECF8CB9F0CF69
:00000001FF
